:020000040000FA
:02000000172EB9
:08000800FF000308FE000A08D6
:10001000FC000408FD008312031300308A00233023
:100020008100A10A063021020318A1012014A20FA9
:100030001C28A30F1C28A0143D08003E03193C28CF
:100040002E1C3A2883160313DB3086008312031319
:10005000860106155B230130652300001E30A400D5
:10006000061107306523061506306523A40B3028DA
:1000700006115E285B233E28502349231430A50037
:10008000FB01FA01EF21F521032254238501210808
:1000900003196920013021020319AA20023021022C
:1000A0000319EB200330210203192C210430210213
:1000B00003196D21053021020319AE210B118B1795
:1000C0007D0884007C088A007E088300FF0E7F0E76
:1000D0000900B830840001080002031C7A17B93007
:1000E000840001080002031CFA167A16BA30840054
:1000F00001080002031CFA15BB308400010800024D
:10010000031C7A15A330840001080002031CFB16AF
:10011000A230840001080002031C7B16FB15A130ED
:10012000840001080002031C7B15A0308400010834
:100130000002031CFB14831603137B0885007A0856
:100140008600831203138030860001308500A50BE2
:1001500069280800BC30840001080002031CFA175B
:10016000BD30840001080002031CFA16BE30840072
:1001700001080002031C7A16FA15BF30840001083A
:100180000002031C7A15A730840001080002031C3A
:10019000FB167B16A630840001080002031CFB1529
:1001A000A530840001080002031C7B15A4308400E4
:1001B00001080002031C7B14831603137B088500CF
:1001C0007A088600831203134030860002308500CF
:1001D000A50BAA280800C030840001080002031CF7
:1001E000FA17C130840001080002031C7A17C230DC
:1001F000840001080002031C7A16C3308400010841
:100200000002031CFA157A15FB16AB3084000108B6
:100210000002031C7B16AA30840001080002031CA4
:10022000FB15A930840001080002031CFB14A83050
:10023000840001080002031C7B14831603137B084F
:1002400085007A088600831203132030860004306C
:100250008500A50BEB280800FA17C43084000108BC
:100260000002031C7A17C530840001080002031C39
:10027000FA16C630840001080002031CFA15C730C4
:10028000840001080002031C7A15AF3084000108C5
:100290000002031CFB16AE30840001080002031CA0
:1002A0007B16AD30840001080002031C7B15AC30C6
:1002B000840001080002031CFB147B148316031343
:1002C0007B0885007A0886008312031310308600AD
:1002D00008308500A50B2C290800C83084000108CF
:1002E0000002031CFA177A17C930840001080002C3
:1002F000031CFA16CA30840001080002031C7A1697
:10030000CB30840001080002031C7A15B33084004E
:1003100001080002031CFB16B23084000108000231
:10032000031CFB15B130840001080002031C7B157F
:10033000FB14B030840001080002031C7B148316F8
:1003400003137B0885007A088600831203130830A4
:10035000860010308500A50B6D290800CC30840084
:1003600001080002031CFA17CD30840001080002C6
:10037000031C7A17FA16CE30840001080002031C11
:100380007A16CF30840001080002031CFA15B7303A
:10039000840001080002031C7B16B63084000108AB
:1003A0000002031CFB157B15B53084000108000218
:1003B000031CFB14B430840001080002031C7B14EE
:1003C000831603137B0885007A08860083120313C3
:1003D0000430860020308500A50BAE2908000310EC
:1003E000260DAF00FC21B20008000310260D013ECF
:1003F000AF00FC21B300080002308A002F08073E3E
:1004000003188A0A820032088A0033088200023404
:1004100047340234523402345A34023462340234DF
:100420006A340234723402347A3402348634023448
:100430008A340234963402349A340234A6340234B4
:10044000AA340234B6340234BA340234C634023424
:10045000CA340234D6340234DA340234E634023494
:10046000EA340234F6340234FA3403340634033402
:100470000A340334163403341A3403342634033470
:100480002A340334363403343A34033446342D10DA
:100490003030B10028184F2A0630A600482B013012
:1004A000A600482B2818572A0030A600482B0230F7
:1004B000A600482B28185F2A0030A600482B0330DE
:1004C000A600482B2818672A0430A600482B0330C2
:1004D000A600482B28186F2A0030A600482B0530AC
:1004E000A600482B2818772A0730A600482B003092
:1004F000A600482B2818842A003031070319822AC5
:10050000B10B482B2D14482BA601482B2808AC0012
:10051000A60A482B2C082806031D902AA601482B62
:1005200028182B10281C2B14A60A482B2808AC00CE
:10053000A60A482B2C082806031DA02AA601482B32
:1005400028182A12281C2A16A60A482B2808AC00AC
:10055000A60A482B2C082806031DB02AA601482B02
:100560002818AA11281CAA15A60A482B2808AC008E
:10057000A60A482B2C082806031DC02AA601482BD2
:1005800028182A11281C2A15A60A482B2808AC006E
:10059000A60A482B2C082806031DD02AA601482BA2
:1005A0002818AA10281CAA14A60A482B2808AC0050
:1005B000A60A482B2C082806031DE02AA601482B72
:1005C00028182A10281C2A14A60A482B2808AC0030
:1005D000A60A482B2C082806031DF02AA601482B42
:1005E0002818A912281CA916A60A482B2808AC000E
:1005F000A60A482B2C082806031D002BA601482B11
:1006000028182912281C2916A60A482B2808AC00ED
:10061000A60A482B2C082806031D102BA601482BE0
:100620002818A911281CA915A60A482B2808AC00CF
:10063000A60A482B2C082806031D202BA601482BB0
:1006400028182911281C2915A60A482B2808AC00AF
:10065000A60A482B2C082806031D302BA601482B80
:100660002818A910281CA914A60A482B2808AC0091
:10067000A60A482B2C082806031D402BA601482B50
:1006800028182910281C2914A60A482BA601301462
:1006900008002D10AD10871E2D14871FAD14080003
:1006A0002810071B2814080027082602031C5A2BB1
:1006B0002608A70008002E10BD030310BC0CBB0CBD
:1006C000BA0CB90C03182E140800B400B40B662B36
:1006D0000800BA01BB01BC01A030B900B709371C42
:1006E0003A143718BA14351E3A15351ABA15B51D0D
:1006F0003A16B519BA16351D3A173519BA17B51C79
:100700003B14B518BB14351C3B153518BB15B61E6C
:100710003B16B61ABB16361E3B17361ABB17B61D4C
:100720003C14B619BC14361D3C153619BC15B61C44
:100730003C16B618BC16361C3C173618BC172130B0
:10074000BD000800BE01BF010830C0000310C20C8C
:10075000BF0DBE0DC10CBF0DBE0DC00BA62B0800FA
:10076000C300C4010830C5000310C30CC40DC50B81
:10077000B42B44080800C6000000C60BBC2B0800C0
:10078000CD0A4D080F3C0319CD014D08B800F90101
:10079000F8010800CD034D08013E031DD22B0E3099
:1007A000CD00B800F901F80108002908CD00B80013
:1007B000F13E031CDF2B0E30CD024D08D82BF90182
:1007C000F8010800C7002010201CE42BC70BE32B06
:1007D00008004D0AB023CF00D001D101D201D301CE
:1007E000D40170305718D000FF30EB24CF01D00176
:1007F000D1010130EB2408000630C8006630C90082
:1008000003104D0DF9008B1359268B17CA000314E2
:100810004D0DF9008B1359268B17C9004A08C800E3
:10082000080021304802031D192C49087907462485
:100830002B2C8B130A08CB0048087807DB00031029
:1008400049087907DC000318DB0A6026CC004B0856
:100850008A004C088B17F90F2E2CF80A0800831613
:1008600003178C18312C8B130C158312031779087E
:100870008D0077088C008316031755308D00AA3041
:100880008D008C148B178312031308008B138316AF
:1008900003178C18492C0C11831203178D00831633
:1008A00003178C130C14831203170C088312031301
:1008B0008B17080000304624D70008005A24571C24
:1008C000632C5710642C57140030F9005708F700B8
:1008D0002F24E923E9230800FC23F901F80111245E
:1008E000CE00CE131124D600D60A1124D800301C15
:1008F000952C07302A02031D802CD523B0016C2CC7
:10090000AA08031D952C203029020319C023213089
:1009100029020319CA23003029020319CD010C3022
:10092000290203195E24B0016C2C2D080319AB2C8D
:10093000E923E92303302D0203195E242D18A32C8B
:10094000AD18A72C6C2CC023E923E9239A2CCA23C9
:10095000E923E9239A2C17304E0204308A00031948
:10096000D82404308A001B304E0208308A00031954
:10097000002804308A003D08003E031DCB2CA01C3B
:10098000CB2CA010571CC62CC0236C2C0730B500F4
:100990003808B6006923D80B772C6C2C590D590DEB
:1009A000591A013AD91A013AD919013AD90008005D
:1009B0001124CF001124D0001124D1001124D20021
:1009C0001124D3001124D4003030DA005608EB246F
:1009D000DA0BE62C0800D500AE3084008001D21B73
:1009E0008009B33084008001521B8009AF3084003D
:1009F0008001D21A8009AB3084008001521A80092C
:100A0000AA3084008001D2198009A23084008001BC
:100A100052198009A33084008001D2188009A730C0
:100A20008400800152188009A63084008001D31B05
:100A30008009A53084008001531B8009A130840007
:100A40008001D31A8009A03084008001531A8009E4
:100A5000B23084008001D3198009B730840080014E
:100A600053198009B63084008001D3188009B13051
:100A70008400800153188009AD3084008001D41BAC
:100A80008009B03084008001541B8009B430840098
:100A90008001D41A8009B53084008001541A80097D
:100AA000AC3084008001D4198009A9308400800111
:100AB00054198009A83084008001D4188009A4301A
:100AC0008400800154188009CC3084008001CF1B41
:100AD0008009C830840080014F1B8009C930840020
:100AE0008001CF1A8009CA30840080014F1A800922
:100AF000CE3084008001CF198009CF30840080017E
:100B00004F198009C13084008001CF188009BC30A2
:100B1000840080014F188009C03084008001D01B00
:100B20008009C43084008001501B8009C5308400D6
:100B30008001D01A8009CD3084008001501A8009CC
:100B4000BB3084008001D0198009BA308400800154
:100B500050198009C33084008001D0188009C63044
:100B60008400800150188009C73084008001D11BA7
:100B70008009CB3084008001511B8009BD30840086
:100B80008001D11A8009B83084008001511A80098F
:100B9000B93084008001D1198009BE308400800101
:100BA00051198009C23084008001D1188009BF30FA
:100BB00084008001511880095508E22308000230A2
:100BC0002602031C0301CF000030D0000130EB24CB
:100BD0002D080319FB2DA701A6013D08003E031DAA
:100BE000E82D2D08D000CF010130EB24B5010C30E9
:100BF000B6006923E82D301CDF2DB001F030CF00A6
:100C0000D0017F30EB24CF01D0013F30EB24F03016
:100C1000CF00D0017F30EB242908CF002A08D00074
:100C2000FF30EB24FF30EB24A701A601DF2D850167
:100C30008101CD01BD01AB01AA01A901AC01A60151
:100C4000A701B001A101A201A301AD018316031305
:100C500071308F04831603178801890183160313EB
:100C60008230810083160313E03087008312031360
:100C7000AD011D30D9008B168B17FF30CF00D0008F
:100C8000D100FF30EB24FF30EB24CF01D001D101A4
:100C9000FF30EB24FF30EB24FF30EB245A242D08E7
:100CA000D000FF30EB24FF30EB242D1C6C2C5E2495
:100CB000DF2D48088A007908490703188A0A82004C
:100CC0000A08CB005B088A005C08820009344734BC
:100CD0000934DA340934EF340A3482340A349D3466
:100CE0000B3430340B3445340B34A8340B34BD345E
:100CF0000B34D2340B34F9340C34B0340D344F345B
:080D00000E343C340E3487343C
:10100000D50004308A001124CF001124D00011240F
:10101000D1001124D2001124D3001124D4000830AF
:101020008A006430BF00AE308400D21B3F21D21F43
:101030004321B3308400521B3F21521F4321AF3064
:101040008400D21A3F21D21E4321AB308400521AB1
:101050003F21521E4321AA308400D2193F21D21DC4
:101060004321A230840052193F21521D4321A33055
:101070008400D2183F21D21C4321A730840052188B
:101080003F21521C4321A6308400D31B3F21D31F94
:101090004321A5308400531B3F21531F4321A1301E
:1010A0008400D31A3F21D31E4321A0308400531A59
:1010B0003F21531E4321B2308400D3193F21D31D59
:1010C0004321B730840053193F21531D4321B630CB
:1010D0008400D3183F21D31C4321B130840053181E
:1010E0003F21531C4321AD308400D41B3F21D41F2A
:1010F0004321B0308400541B3F21541F4321B4309E
:101100008400D41A3F21D41E4321B5308400541AE0
:101110003F21541E4321AC308400D4193F21D41DFB
:101120004321A930840054193F21541D4321A83084
:101130008400D4183F21D41C4321A43084005418C7
:101140003F21541C4321CC308400CF1B3F21CF1FB3
:101150004321C83084004F1B3F214F1F4321C9301A
:101160008400CF1A3F21CF1E4321CA3084004F1A7A
:101170003F214F1E4321CE308400CF193F21CF1D88
:101180004321CF3084004F193F214F1D4321C130EF
:101190008400CF183F21CF1C4321BC3084004F185E
:1011A0003F214F1C4321C0308400D01B3F21D01F62
:1011B0004321C4308400501B3F21501F4321C530C0
:1011C0008400D01A3F21D01E4321CD308400501A14
:1011D0003F21501E4321BB308400D0193F21D01D38
:1011E0004321BA30840050193F21501D4321C330A0
:1011F0008400D0183F21D01C4321C63084005018F1
:101200003F21501C4321C7308400D11B3F21D11FF7
:101210004321CB308400511B3F21511F4321BD305E
:101220008400D11A3F21D11E4321B8308400511AC5
:101230003F21511E4321B9308400D1193F21D11DD6
:101240004321BE30840051193F21511D4321C2303A
:101250008400D1183F21D11C4321BF308400511894
:101260003F21511C4321550803308A00E2230830F6
:101270008A00BF0B1328831304308A00BB2C800A1A
:101280000319800908008008031D80030800173433
:101290001034183480340034003480340034003486
:1012A00040340034003440340034003420340034FE
:1012B000003420340034003410340034003410344E
:1012C000003400340834003400340834003400346E
:1012D0000434003400340434003400340234003464
:1012E000003402340034003401340034003401345A
:1012F000003400340034803400340034803400344E
:10130000003440340034003440340034003420349D
:1013100000340034203400340034103400340034FD
:1013200010340034003408340034003408340034FD
:101330000034043400340034043400340034023403
:1013400000340034023400340034013400340034FA
:1013500001340034003400348034003400348034EC
:10136000003400344034003400344034003400345D
:10137000203400340034203400340034103400347D
:10138000003410340034003408340034003408349D
:1013900000340034043400340034043400340034A5
:1013A0000234003400340234003400340134003498
:1013B00000340134173410340334FF34FF34FF3465
:1013C000FF34FF34FF34FF34F0340034FF34F034A2
:1013D000003400340F34FF3400340F34FF3417343A
:1013E0000334183480341034003480341034003422
:1013F000403420340034403420340034203440342D
:10140000003420344034003410348034003410343C
:10141000803400340934003400340934003400349A
:101420000634003400340634003400348034103480
:1014300000348034103400344034203400344034DC
:10144000203400342034403400342034403400341C
:1014500010348034003410348034003409340034C3
:1014600000340934003400340634003400340634C7
:1014700000340034003408340134003408340134BA
:1014800000340434023400340434023400340234AE
:101490000434003402340434003401340834003499
:1014A0000134083400340034903400340034903473
:1014B00000340034603400340034603400340834C4
:1014C000013400340834013400340434023400346C
:1014D000043402340034023404340034023404345A
:1014E000003401340834003401340834003400344A
:1014F00090340034003490340034003460340034CC
:1015000000346034173410340434FC340F34C034E5
:10151000003400340034003400340034FC340F3420
:10152000C0340334F0343F34003400340034003429
:10153000003400340334F0343F341B341034183496
:10154000FF34FF34FF34FF34FF34FF34FF34FF3403
:10155000FF34FF34FF34FF34FF34FF34FF34FF34F3
:10156000FF34FF34FF34FF34FF34FF34FF34FF34E3
:1015700000340034003400340034003400340034CB
:1015800000340034003400340034003400340034BB
:1015900000340034003400340034003400340034AB
:1015A000FF34F0340034FF34F0340034FF34F034CE
:1015B0000034FF34F0340034FF34F0340034FF34AE
:1015C000F0340034FF34F0340034FF34F0340034AD
:1015D000003400340034003400340034003400346B
:1015E000003400340034003400340034003400345B
:1015F000003400340034003400340034003400344B
:1016000000340F34FF3400340F34FF3400340F340F
:10161000FF3400340F34FF3400340F34FF3400340F
:101620000F34FF3400340F34FF3400340F34FF34F0
:10163000003400340034003400340034003400340A
:1016400000340034003400340034003400340034FA
:1016500000340034003400340034003400340034EA
:10166000173403340334DB346D34B634DB346D3477
:10167000B6346D34B634DB346D34B634DB34B63462
:10168000DB346D34B634DB346D341734023410344B
:10169000803410340034803410340034403420342A
:1016A0000034403420340034A03450340034A034AA
:1016B000503400345034A03400345034A03400345A
:1016C0002934403400342934403400341634803412
:1016D00000341634803400340934003400340934C2
:1016E000003400340634003400340634003400344E
:1016F0000034083401340034083401340034043434
:10170000023400340434023400340A340534003422
:101710000A340534003405340A34003405340A34FC
:1017200000340234943400340234943400340134EC
:1017300068340034013468340034003490340034A8
:1017400000349034003400346034003400346034A9
:10175000173403340334DB3460340034DB34603456
:1017600000346D34B03400346D34B0340034B634E9
:10177000D03400346D34B0340034173403340334BF
:1017800000340D34B63400340D34B634003406342D
:10179000DB3400340634DB3400340B346D34003475
:1017A0000B346D34173403340634C33401348634B7
:1017B000C3340134863461348034C33461348034BA
:1017C000C3343034C83461343034C83461341834EC
:1017D0006C34303418346C3430340C3436341834BF
:1017E0000C3436341834863413340C3486341334C1
:1017F0000C341B3403341E34803400340134003480
:1018000000340034C0340034033400340034003475
:10181000E03400340734003400340034F034003451
:101820000F34003400340034783400341E34003473
:10183000003400343C3400343C3400340034003490
:101840001E34003478340034003400340F34003453
:10185000F03400340034003407348134E034003490
:10186000003400340334C334C03400340034003452
:101870000134E73480340034003400340034FF3461
:10188000003400340034003400347E34003400343A
:101890000034003400343C3400340034003400346C
:1018A0000034183400340034003400340034003480
:1018B0000034803400340134003400340034C03447
:1018C00000340334003400340034E034003407348E
:1018D000003400340034F03400340F340034003469
:1018E0000034783400341E340034003400343C3486
:1018F00000343C340034003400341E340034783476
:101900000034003400340F340034F0340034003438
:10191000003407348134E0340034003400340334BC
:10192000C334C0340134003400340134E73480342B
:101930000034003400340034FF3400340034003408
:10194000003400347E340034003400340034003479
:101950003C34003400340034003400341834003493
:101960001B3403341A34803410340034803410347F
:101970000034C03430340034C03430340034E03407
:1019800070340034E03470340034F034F034003417
:10199000F034F03400347934E03400347934E03415
:1019A00000343F34C03400343D34C03400341F347C
:1019B000803400341F34803400340F340034003459
:1019C0000F3400340034063400340034063400345C
:1019D0000034003400340034003400340034003467
:1019E0000034003400340034003400340034003457
:1019F0000034003400340034003400340034003447
:101A00000034003408340134003408340134003424
:101A10000C34033400340C34033400340E340734F3
:101A200000340E34073400340F340F3400340F34D4
:101A30000F34003407349E34003407349E340034AD
:101A40000334FC3400340334FC3400340134F834FF
:101A500000340134F83400340034F03400340034FD
:101A6000F034003400346034003400346034003426
:101A700000340034003400340034003400340034C6
:101A800000340034003400340034003400340034B6
:101A900000340034003400340034003400341B348B
:101AA0000334273406340034003406340034003460
:101AB0000F34003400340F34003400341F348034C9
:101AC00000341F34803400343F34C03400343D349B
:101AD000C03400347934E03400347934E0340034F4
:101AE000F034F0340034F034F0340034E034703446
:101AF0000034E03470340034C03430340034C03446
:101B000030340034803410340034803410340034E5
:101B10000034003400340034003400340034003425
:101B20000034003400340034003400340034003415
:101B30000034003400340034003400340034003405
:101B40000034003460340034003460340034003435
:101B5000F03400340034F03400340134F83400340C
:101B60000134F83400340334FC3400340334FC34DE
:101B7000003407349E34003407349E3400340F346C
:101B80000F3400340F340F3400340E340734003473
:101B90000E34073400340C34033400340C34033472
:101BA0000034083401340034083401340034003483
:101BB0000034003400340034003400340034003485
:101BC0000034003400340034003400340034003475
:101BD000003400340034003400340034063400345F
:101BE00060340634003460340F340034F0340F3481
:101BF0000034F0341F348134F8341F348134F83425
:101C00003F34C334FC343F34C334FC347934E734D8
:101C10009E347934E7349E34F034FF340F34F0349A
:101C2000FF340F34E0347E340734E0347E3407343C
:101C3000C0343C340334C0343C340334803418346E
:101C4000013480341834013400340034003400345A
:101C500000340034003400340034003400340034E4
:101C600000340034003400340034003400340034D4
:101C70000034003400340034173403340C3480341E
:101C800010340034803410340034203440340034B4
:101C90002034403400340934003400340934003432
:101CA0000034003408340134003408340134003482
:101CB00002340434003402340434003400349034E8
:101CC0000034003490344034203400344034203424
:101CD000003410348034003410348034003406343E
:101CE0000034003406340034003400340434023448
:101CF0000034043402340034013408340034013434
:101D00000834003400346034003400346034173454
:101D100001342134C03430340034C0343034003421
:101D2000003400340034003400340034C034303423
:101D30000034C03430340034003400340034003413
:101D40000034003400340C34033400340C340334D5
:101D500000340034003400340034003400340C34D7
:101D6000033400340C3403340034003400340034C1
:101D700000340034003400340034003400340034C3
:101D800000340034003400340034003400340034B3
:101D900000340034003400343034C0340034303483
:101DA000C0340034003400340034003400340034D3
:101DB0003034C03400343034C034003400340034A3
:101DC0000034003400340034003403340C34003464
:101DD00003340C3400340034003400340034003454
:101DE000003403340C34003403340C340034003435
:101DF0000034003400340034003400340034003443
:101E00000034003400340034003400340034003432
:101E10000034003400340034003400340F34003413
:101E200000340F3400340034003400340034003403
:101E3000003400340F34003400340F3400340034E4
:101E400000340034003400340034003400340034F2
:101E5000F03400340034F034003400340034003402
:101E60000034003400340034F03400340034F034F2
:101E700000340034003400340034003400340034C2
:101E800000340034003400340034003400340034B2
:101E900000340034003400340034003400340034A2
:02400E00C428C4
:02401000FF3E71
:02420000FF3489
:00000001FF
